:1000000019C033C032C031C030C02FC02EC02DC087
:100010002CC02BC02AC029C028C027C026C025C09C
:1000200024C023C022C021C020C01FC01EC01DC0CC
:100030001CC01BC011241FBECFEFD4E0DEBFCDBF5C
:1000400011E0A0E0B1E0EEEDF2E002C005900D920B
:10005000AE30B107D9F721E0AEE0B1E001C01D92AA
:10006000A431B207E1F7E0D038C1CACF8FEF8AB927
:1000700087E084B93B9843982FEF81E19AE72150BC
:1000800080409040E1F700C0000008951BB884E074
:1000900085B986E08A95F1F700C0E0911301F0E0A0
:1000A000E050FF4F80818BB987E893E10197F1F72A
:1000B00000C000001BB882E085B996E09A95F1F780
:1000C00000C0E0911201F0E0E050FF4F80818BB959
:1000D00087E893E10197F1F700C000001BB881E0C9
:1000E00085B996E09A95F1F700C08DEA8BB987E85B
:1000F00093E10197F1F700C0000008950F931F935B
:10010000CF93DF9300D000D01F92CDB7DEB73B98DE
:1001100089EC07C036E03A95F1F700C0815009F448
:100120006EC03399F7CF86E507C096E09A95F1F750
:1001300000C0815009F465C0339BF7CF86E507C046
:10014000A6E0AA95F1F700C0815009F45CC033998C
:10015000F7CFFE01319685E0DF011D928A95E9F720
:10016000AE014A5F5F4F22C0B6E0BA95F1F700C01A
:10017000915011F44AC098E3339BF6CF38EC3A958E
:10018000F1F7220F339908C00BC0A6E0AA95F1F74A
:1001900000C0915011F43BC09EE23399F6CF21602C
:1001A000815049F721934E175F0719F088E020E04E
:1001B000E2CFA981B0E0EA81F0E06B8170E04C8190
:1001C00050E09D012E0F3F1F260F371F240F351FB4
:1001D00033270D8110E020173107D9F4BA2FAA2751
:1001E000EA0FFB1FF0931101E0931001762F6627B1
:1001F000460F571F50930F0140930E010BC082E032
:1002000009C083E007C084E005C085E003C086E044
:1002100001C087E00F900F900F900F900F90DF912B
:10022000CF911F910F91089521DF8AE080931301F0
:100230008BE080931201C0E0D0E01CE03AC0339B19
:1002400002C03B9A4398CE3E83E0D80790F156DF38
:10025000811129C0E0911001F09111019F01ADECD5
:10026000BCEC2FD0AC0156954795569547955695C1
:100270004795509311014093100136952795369577
:100280002795ABE7B4E11DD0969587958093130130
:10029000880F982F990F990F890F481B40931201CF
:1002A000C0E0D0E006C01093130180931201C0E0BB
:1002B000D0E02196EBDEC93E83E0D80708F0BFCF3F
:1002C000F8CFA29FB001B39FC001A39F01D0B29FFE
:0E02D000700D811D1124911D0895F894FFCF2B
:0E02DE00FC24BAAE66CEDEA4FEEE161EDA12C8
:00000001FF
